:100000000C94E2050C940A060C940A060C940A0659
:100010000C940A060C940A060C940A060C940A0620
:100020000C940A060C940A060C94AC070C941E0857
:100030000C940A060C940A060C940A060C940A0600
:100040000C940A060C94450D0C940A060C940A06AE
:100050000C940A060C940A060C940A060C94580C8C
:100060000C940A060C940A060C940A060C940A06D0
:100070000C940A060C940A060C940A060C940A06C0
:100080000C94E30D0C940A060C940A060C940A06D0
:100090000C940A060C940A060C940A060C940A06A0
:1000A0000C940A060C940A060C940A0615148B1478
:1000B000ED1426158F15CA15A8164417FF17B0188A
:1000C000EA183D196119AA19D119860A890A780A0C
:1000D0007C0A800AAA0AAA0AAA0A8D0A910A950A23
:1000E0009B0A9F0AAA0AA50A210B260B2B0B350B8C
:1000F0003F0B890B890B890B490B530B5D0B670B6E
:10010000740B890B7C0BF0F89C8E8783878E9CF890
:10011000F00000FEFF0303030303070EFCF80000DA
:10012000FEFF0303030303070EFCF80000FFFF00BC
:10013000000000000000FFFF0000FEFF83838383B8
:1001400083C7EE7C380000F8FC0E07030303070E9C
:10015000FCF800003F7FE0C08080C0E07F3FFFFFF1
:1001600001010101010101FFFF0000FFFF0C0C0C68
:100170000C1C3E77E3C100007FFFC0C0C0C0C0E0E0
:10018000703F1F00001F3F70E0C0C0C0E0703F1F05
:1001900000007FFFC1C1C1C1C1E3773E1C00001F49
:1001A0003F70E0C0C0C0E0703F1F000000000001D1
:1001B000FFFF0100000000000000240027002A00CB
:1001C0002D003000D5F08D14A1C881CFD9F1AF201A
:1001D0000014021302120215020702080204010CA5
:1001E00001060100687474703A2F2F7777772E63B9
:1001F000726169742E6E65742F0040637261697458
:10020000004A6F6E617468616E20486F6C6D657333
:100210000041726475626F79204173736973746110
:100220006E7420312E3100436F6E6E6563742079D9
:100230006F75722041726475626F790A746F2079EC
:100240006F757220636F6D707574657220616E6476
:100250000A72756E207468652041726475696E6FEC
:100260002049444527730A73657269616C206D6F7C
:100270006E69746F722E0A0A436861722052656358
:1002800065697665643A2000284129205965732004
:100290002D20284229204E4F0052656365697669FA
:1002A0006E672E2E2E00596F757220454550524FA5
:1002B0004D2077696C6C2062650A657261736564B4
:1002C00020666F7220676F6F64207768656E0A72B0
:1002D0006573746F72696E6720454550524F4D20AB
:1002E00066726F6D0A7468652041726475696E6F1D
:1002F000204944452E204172650A796F7520737537
:1003000072653F0A0028412920596573202D202855
:100310004229204E4F00596F757220454550524F6B
:100320004D2077696C6C2062650A65726173656443
:1003300020666F7220676F6F642E204172650A79A4
:100340006F75207375726520796F752077616E7493
:1003500020746F0A646F20746869733F0028412914
:1003600020596573202D20284229204E4F00436FCD
:100370006E6E65637420796F757220417264756268
:100380006F790A746F20796F757220504320616E07
:10039000642072756E0A7468652041726475696EB6
:1003A0006F204944452E0A002855702F446F776E00
:1003B00029204672657175656E63790A2841292086
:1003C000506C6179202D20284229204261636B0006
:1003D00028412920546F67676C65202D2028422909
:1003E000204261636B0020202056696577204545D7
:1003F00050524F4D0A2020204261636B2D557020D2
:10040000454550524F4D0A202020526573746F723B
:100410006520454550524F4D0A202020436C6561B0
:100420007220454550524F4D002855702F446F772C
:100430006E29205363726F6C6C0A28422920426136
:10044000636B00427574746F6E20546573740A2078
:10045000202043686172616374657220546573740F
:100460000A202020454550524F4D204D616E616756
:1004700065720A2020204C454420546573740A207C
:10048000202053637265656E20546573740A2020C2
:1004900020536F756E6420546573740A20202055B4
:1004A0005342205472616E73666572205465737492
:1004B0000A20202041626F757400687474703A2FAE
:1004C0002F7777772E63726169742E6E65742F00B3
:1004D000406372616974004A6F6E617468616E2076
:1004E000486F6C6D65730041726475626F7920416D
:1004F0007373697374616E7420312E3100000000D3
:1005000000003E5B4F5B3E3E6B4F6B3E1C3E7C3EB5
:100510001C183C7E3C181C577D571C1C5E7F5E1CC3
:1005200000183C1800FFE7C3E7FF0018241800FF7D
:10053000E7DBE7FF30483A060E2629792926407F77
:10054000050507407F05253F5A3CE73C5A7F3E1C86
:100550001C08081C1C3E7F14227F22145F5F005F72
:100560005F06097F017F006689956A606060606050
:1005700094A2FFA29408047E040810207E20100894
:10058000082A1C08081C2A08081E101010100C1E2F
:100590000C1E0C30383E3830060E3E0E06000000B1
:1005A000000000005F00000007000700147F147FB8
:1005B00014242A7F2A1223130864623649562050D5
:1005C0000008070300001C2241000041221C002AF1
:1005D0001C7F1C2A08083E080800807030000808AC
:1005E000080808000060600020100804023E51491D
:1005F000453E00427F400072494949462141494DEC
:10060000331814127F1027454545393C4A49493172
:1006100041211109073649494936464949291E00F1
:10062000001400000040340000000814224114149B
:10063000141414004122140802015909063E415DB8
:10064000594E7C1211127C7F494949363E41414145
:10065000227F4141413E7F494949417F09090901C2
:100660003E414151737F0808087F00417F410020CF
:1006700040413F017F081422417F404040407F02BB
:100680001C027F7F0408107F3E4141413E7F0909E3
:1006900009063E4151215E7F0919294626494949EB
:1006A0003203017F01033F4040403F1F2040201F95
:1006B0003F4038403F631408146303047804036127
:1006C00059494D43007F4141410204081020004137
:1006D00041417F04020102044040404040000307C2
:1006E000080020545478407F284444383844444417
:1006F00028384444287F385454541800087E09028E
:1007000018A4A49C787F0804047800447D4000204D
:1007100040403D007F1028440000417F40007C04A1
:100720007804787C080404783844444438FC18245D
:10073000241818242418FC7C080404084854545431
:100740002404043F44243C4040207C1C2040201CC6
:100750003C4030403C44281028444C9090907C44CD
:1007600064544C440008364100000077000000410A
:1007700036080002010204023C2623263C1EA1A1E9
:1007800061123A4040207A385454555921555579D0
:100790004121545478412155547840205455794092
:1007A0000C1E5272123955555559395454545939F1
:1007B000555454580000457C410002457D420001DB
:1007C000457C40F0292429F0F0282528F07C545558
:1007D00045002054547C547C0A097F4932494949D8
:1007E000323248484832324A4848303A4141217A08
:1007F0003A42402078009DA0A07D39444444393DD0
:100800004040403D3C24FF2424487E4943662B2F32
:10081000FC2F2BFF0929F620C0887E0903205454A1
:1008200079410000447D413048484A3238404022F6
:100830007A007A0A0A727D0D19317D2629292F281E
:10084000262929292630484D40203808080808085C
:10085000080808382F10C8ACBA2F102834FA000046
:100860007B000008142A142222142A14089500225E
:100870000095AA005500AAAA55AA55AA000000FF93
:1008800000101010FF00141414FF001010FF00FFE0
:100890001010F010F0141414FC001414F700FF00F2
:1008A00000FF00FF1414F404FC141417101F1010A0
:1008B0001F101F1414141F00101010F0000000006F
:1008C0001F101010101F10101010F010000000FF6B
:1008D000101010101010101010FF10000000FF1466
:1008E0000000FF00FF00001F10170000FC04F414BC
:1008F000141710171414F404F40000FF00F7141474
:100900001414141414F700F7141414171410101FEF
:10091000101F141414F4141010F010F000001F1025
:100920001F0000001F14000000FC140000F010F075
:100930001010FF10FF141414FF141010101F0000EB
:100940000000F010FFFFFFFFFFF0F0F0F0F0FFFFFE
:10095000FF0000000000FFFF0F0F0F0F0F3844448F
:1009600038447C2A2A3E147E02020606027E027E5B
:100970000263554941633844443C04407E201E20B4
:1009800006027E020299A5E7A5991C2A492A1C4C59
:100990007201724C304A4D4D303048784830BC625C
:1009A0005A463D3E494949007E0101017E2A2A2AD4
:1009B0002A2A44445F444440514A444040444A51F6
:1009C000400000FF0103E080FF000008086B6B0897
:1009D0003612362436060F090F06000018180000DC
:1009E000001010003040FF0101001F01011E00191E
:1009F0001D1712003C3C3C3C0000000000060115A5
:100A000001260137014A015D01720188019F01B889
:100A100001D201EE010B022A024B026E029302BACE
:100A200002E40210033F037003A403DC0317045520
:100A3000049704DD0427057505C80520067D06E03A
:100A4000064907B8072D08A9082D09B9094D0AEA72
:100A50000A900B400CFA0CC00D910E6F0F5A1053F8
:100A6000115B1272139A14D41520178018F519808F
:100A70001B231DDE1EB420A622B524E4263429A79C
:100A80002B402E0031EA330037453ABC3D68414CDB
:100A9000456B49C84D68524F57805C006210111277
:100AA00013151617181A1C1D1F21232527292C2E54
:100AB0003134373A3E4145494E52575C62686E7553
:100AC0007B838B939CA5AFB9C4D0DCE9F700000011
:100AD0000200090F0000030401000C0000000000E8
:100AE000000000000000000000000000080B0002F1
:100AF00002020100090400000102020000052400B6
:100B00001001052401010104240206052406000148
:100B10000705810310004009040100020A000000DB
:100B2000070502024000000705830240000004039D
:100B3000090441726475696E6F204C4C4300417228
:100B40006475696E6F204C656F6E6172646F001220
:100B50000100020000004041233680000101020331
:100B60000112010002EF0201404123368000010121
:100B70000203010408020110408040102040804020
:100B800080080204018040201002011080102040E3
:100B9000402000000000250028002B002E0031001E
:100BA0000404040404030405020202020403020212
:100BB00002020606060606060404020202040403F4
:100BC00001004F1C11241FBECFEFDAE0DEBFCDBF06
:100BD00027E0A2EDB2E001C01D92AE39B207E1F705
:100BE00012E0A0E0B1E0EAE9FFE302C005900D9257
:100BF000A23DB107D9F715E0C2EED5E004C02197B8
:100C0000FE010E94821CC13ED107C9F70E947011EB
:100C10000C94CB1F0C94000040911A0350911B03BD
:100C2000209118033091190342175307B4F490919F
:100C3000E8009570E1F39091E80092FD19C080936F
:100C4000F10080911A0390911B0301968F739927ED
:100C5000892B19F48EEF8093E80080911A0390910C
:100C60001B03019690931B0380931A0381E0089560
:100C700080E00895CF92DF92EF92FF920F931F933F
:100C8000CF93DF931F92CDB7DEB7182F062FE42E38
:100C9000862F880F8E5F99830E940C0683E00E9446
:100CA0000C06F12EC12E9981D92E8C2D8F1980170B
:100CB00098F4F601E7FE02C0849101C080810E9491
:100CC0000C06182F80E00E940C068123FFEFCF1A3C
:100CD000DF0A8111EACF01C081E00F90DF91CF914F
:100CE0001F910F91FF90EF90DF90CF900895DF92CA
:100CF000EF92FF920F931F93CF93DF93D82E8A0129
:100D00007B01E40EF51EEB01CE15DF0571F0D7FE79
:100D100003C0FE01849101C088810E940C062196C7
:100D20008111F2CF8FEF9FEF01C0C801DF91CF910A
:100D30001F910F91FF90EF90DF900895615030F078
:100D40002091F100FC0120830196F8CF289884E6D9
:100D500080931D030895CF92DF92EF92FF920F933D
:100D60001F93CF93DF936C017A018B01C0E0D0E039
:100D7000CE15DF0589F0D8016D918D01D601ED9179
:100D8000FC910190F081E02DC6010995892B11F4A9
:100D90007E0102C02196ECCFC701DF91CF911F9158
:100DA0000F91FF90EF90DF90CF900895CF93DF9356
:100DB0001F92CDB7DEB76983DC01ED91FC91028013
:100DC000F381E02D41E050E0BE016F5F7F4F099558
:100DD0000F90DF91CF91089583E08093E900809197
:100DE000F200882319F08AE38093E8000895FC015B
:100DF0008485958597FD0BC09FB7F89482E080931A
:100E0000E9008091F2009FBF90E0019608959FB79E
:100E1000F89482E08093E9008091F2009FBF90E017
:100E200008953FB7F8948091130390911403A09113
:100E30001503B091160326B5A89B05C02F3F19F0E6
:100E40000196A11DB11D3FBFBA2FA92F982F88274A
:100E5000820F911DA11DB11DBC01CD0142E0660FA5
:100E6000771F881F991F4A95D1F708950E94881C03
:100E70000F931F93CF93DF931F92CDB7DEB782E01E
:100E8000898342E450E06CEE7AE080E80E947706C5
:100E90000E945C11DC0112960D911C9113970115B3
:100EA000110569F0D801ED91FC910280F381E02DEC
:100EB000BE016F5F7F4FC801099597FF07C0898109
:100EC0000F90DF91CF911F910F910895F801008548
:100ED0001185E5CFCF93DF931F92CDB7DEB7FC012D
:100EE0008485958597FD05C02FEF3FEF35872487D3
:100EF0000BC0CE0101960E943211019719F489812D
:100F000090E002C08FEF9FEF0F90DF91CF91089597
:100F10000F931F93CF93DF931F92CDB7DEB78C0152
:100F2000FC018485958597FF0EC0CE0101960E9435
:100F30003211019719F4298130E002C02FEF3FEF01
:100F4000F80135872487F801848595850F90DF9116
:100F5000CF911F910F9108951F920F920FB60F928C
:100F600011248F939F938091E1009091E100937FF2
:100F70009093E10083FF0FC01092E90091E09093FD
:100F8000EB001092EC0092E39093ED0010921E03A0
:100F900098E09093F00082FF20C093E09093E900E6
:100FA0009091F200992319F09AE39093E8009091C0
:100FB0001C03992339F090911C03915090931C03CA
:100FC000992389F190911D03992339F090911D0384
:100FD000915090931D03992341F184FF10C080919B
:100FE000E2008E7E81608093E2008091E1008F7E3E
:100FF0008093E1008091D3028E7E806111C080FFDA
:1010000016C08091E2008E7E80618093E200809124
:10101000E1008E7E8093E1008091D3028E7E81601C
:101020008093D30204C05D9ACDCF289AD6CF9F91EA
:101030008F910F900FBE0F901F9018951F920F92D7
:101040000FB60F921124CF92DF92EF92FF920F937F
:101050001F932F933F934F935F936F937F938F9340
:101060009F93AF93BF93EF93FF93CF93DF93CDB74E
:10107000DEB76C97DEBFCDBF1092E9008091E8002B
:1010800083FFFAC168E0CE0145960E949E0682EF7A
:101090008093E8008D8987FF05C09091E80090FF5C
:1010A000FCCF03C09EEF9093E800982F907609F054
:1010B000C6C09E892F89188D91110CC0803829F4E3
:1010C0008091D4028093F10002C01092F10010923E
:1010D000F10047C1422F50E0512B913051F4811162
:1010E00040C14130510509F03CC18091D4028D7F4F
:1010F0000BC0933061F4811134C14130510509F0C6
:1011000030C18091D40282608093D4022AC195308C
:1011100041F48091E80080FFFCCF20682093E30039
:1011200020C1963009F05FC0EB8CFC8C1092E90076
:1011300010921B0310921A03123091F510921903AA
:10114000109218030E94380799E0BE016F5F7F4F2D
:10115000DB01E92F1D92EA95E9F799831A8391E063
:101160009E8390EA98879AEF998720911A0330918D
:101170001B03275F3F4F3C832B838D831092E90035
:1011800010921B0310921A03F0921903E0921803B5
:1011900049E050E080E00E9477060E943807E1C0F5
:1011A000F0921903E09218030E945C11DC01129680
:1011B000ED90FC901397E114F10409F4C0C0D7013D
:1011C000ED91FC910480F581E02DBE016B5E7F4FB7
:1011D000C7010995009719F00CF0C3C0C6C0F7010C
:1011E000E084F184E8CF973009F4BFC0983021F44F
:1011F00081E08093F100B5C0993009F0B2C08370EE
:1012000009F0B3C0E4E2F1E081E021E036E390814F
:10121000992361F08093E9002093EB0091919093E2
:10122000EC003093ED008F5F873089F78EE7809375
:10123000EA001092EA008F8980931E0392C08B8D82
:101240009C8D1092E90010921B0310921A03909348
:10125000190380931803898D811156C08E899D8949
:10126000913A59F4813209F080C047E050E067E1DB
:1012700071E080E00E94770674C0913209F075C079
:10128000833289F4888D90E0982F88272F89822BCC
:10129000A0E0B0E08093130190931401A093150196
:1012A000B09316015EC0803269F48091E80082FF3D
:1012B000FCCF67E087E191E00E949E068BEF809370
:1012C000E80006C0823209F04CC08F8980931E016D
:1012D0008091D202882319F0EEEFFAE002C0E0E03C
:1012E000F8E08091170190911801A0911901B09137
:1012F0001A01803B9440A105B10509F088C0809196
:101300001E0180FFA0C083C00E945C11DC01129608
:101310000D911C9113970115110539F1D801ED912B
:10132000FC910190F081E02DBE016B5E7F4FC80102
:101330000995811116C0F80100851185ECCF113097
:10134000C1F0133091F48F89882309F455C082309D
:10135000E9F440E860E18EE39BE00E943A068823CE
:1013600021F08EEF8093E80087C081E28093EB004C
:1013700083C08B8D9C8D089711F410931703809177
:101380001703811136C06FE47BE038C0813029F447
:1013900040E86BE082E39BE0E0CF833031F70E94CE
:1013A0005C11DC011296ED90FC9013978E010F5F9B
:1013B0001F4F6801E114F10479F0D701ED91FC9120
:1013C0000680F781E02DB801C7010995080F111DAE
:1013D000F701E084F184EECFD8011C92F601019070
:1013E0000020E9F73197BF016C197D0940E0C60183
:1013F000B4CF61E67BE002C06EE27BE0611571056F
:1014000009F4B3CFFB01449150E080E833CF0FB62D
:10141000F894A89580916000886180936000109294
:1014200060000FBEA895EE3F2AE0F20739F08091E8
:10143000FE0A9091FF0A9183808393CF1092FF0A56
:101440001092FE0A8ECFEE3F8AE0F80731F08081DD
:1014500091819093FF0A8093FE0A87E797E7918333
:1014600080839BE088E10FB6F894A8958093600094
:101470000FBE9093600075CF6C960FB6F894DEBFE8
:101480000FBECDBFDF91CF91FF91EF91BF91AF9193
:101490009F918F917F916F915F914F913F912F918C
:1014A0001F910F91FF90EF90DF90CF900F900FBEA4
:1014B0000F901F901895362F90E0FC01E353F54FE5
:1014C0004491FC01ED58F44F2491FC01E056F44F97
:1014D0008491882309F451C04423E1F150E0FA01DA
:1014E0003197EF30F105B0F5EB59FF4F0C94821CAA
:1014F000909180009F7707C0909180009F7D03C0EE
:1015000090918000977F9093800024C094B59F773E
:1015100002C094B59F7D94BD1DC0909190009F77AF
:1015200007C0909190009F7D03C090919000977F9D
:10153000909390000FC09091C0009F7703C090914E
:10154000C0009F7D9093C00005C09091C200977F1E
:101550009093C200E82FF0E0EE0FFF1FEE56F44F1D
:10156000A591B4918FB7F894EC91311103C02095F7
:101570002E2301C02E2B2C938FBF0895CF93DF9382
:1015800090E0FC01ED58F44F2491FC01E056F44F3B
:101590008491882361F190E0880F991FFC01EA543F
:1015A000FE4FC591D491FC01EE56F44FA591B49134
:1015B000611109C09FB7F8948881209582238883A0
:1015C000EC912E230BC0623061F49FB7F894388100
:1015D000822F809583238883EC912E2B2C939FBFA1
:1015E00006C08FB7F894E8812E2B28838FBFDF9138
:1015F000CF9108951F93CF93DF93182FEB0161E0F4
:101600000E94BE0A209711F460E004C0CF3FD105CC
:1016100039F461E0812FDF91CF911F910C945B0A27
:10162000E12FF0E0E353F54FE4914E2F50E0FA0143
:101630003197EF30F10508F06CC0EC58FF4F0C9477
:10164000821C84B5806884BDC7BD68C084B58062D3
:1016500084BDC8BD63C08091800080688093800095
:10166000D0938900C093880059C080918000806227
:1016700080938000D0938B00C0938A004FC08091EC
:101680008000886080938000D0938D00C0938C0090
:1016900045C080919000806880939000D09399001D
:1016A000C09398003BC0809190008062809390002E
:1016B000D0939B00C0939A0031C0809190008860C5
:1016C00080939000D0939D00C0939C0027C0809190
:1016D000C00080688093C0008091C0008F7B8093A1
:1016E000C000C093CF001AC08091C0008062809378
:1016F000C000C093D00012C08091C2008860809367
:10170000C2008091C2008B7F8093C200C093D20040
:1017100005C0C038D1050CF07CCF76CFDF91CF91DA
:101720001F9108958F929F92AF92BF92CF92DF92B6
:10173000EF92FF926B017C010E9411074B015C014B
:10174000C114D104E104F104F1F00E941107DC019D
:10175000CB0188199909AA09BB09883E9340A105C4
:10176000B10570F321E0C21AD108E108F10888EE52
:10177000880E83E0981EA11CB11CC114D104E104A1
:10178000F10419F7DDCFFF90EF90DF90CF90BF907D
:10179000AF909F908F9008958F929F92AF92BF923B
:1017A000CF92DF92EF92FF920F931F93CF93DF932D
:1017B0005C016B018A0180911E01882309F45EC0DF
:1017C00080911E03882309F459C08091D30280FFC1
:1017D00005C08091E00082608093E000E8018AEF1C
:1017E000F82E93E0E92E2FE3822E3AE3932E2097F2
:1017F00009F43DC08FB7F894E092E9009091E800B9
:1018000095FF06C09091F200282D291B922F01C050
:1018100090E08FBF91110AC0FA94FF2079F161E046
:1018200070E080E090E00E94920BE1CF292F30E041
:10183000C217D3070CF49C2F8FB7F894E092E900FD
:101840002091E80025FF11C0292F30E0C21BD30BE7
:10185000F601915020F041914093F100FACFC20E71
:10186000D31E9091E80095FF13C08FBFC0CF5D9845
:1018700084E680931C031016110644F081E090E08A
:10188000F5019383828380E090E005C0C80103C026
:101890009092E800EACFDF91CF911F910F91FF90D6
:1018A000EF90DF90CF90BF90AF909F908F90089572
:1018B0001F920F920FB60F9211242F933F938F9385
:1018C0009F93AF93BF9380910F0390911003A091CA
:1018D0001103B091120330910E0323E0230F2D3733
:1018E00020F40196A11DB11D05C026E8230F029624
:1018F000A11DB11D20930E0380930F03909310033D
:10190000A0931103B09312038091130390911403D9
:10191000A0911503B09116030196A11DB11D8093EE
:10192000130390931403A0931503B0931603BF9170
:10193000AF919F918F913F912F910F900FBE0F907C
:101940001F9018958FB12CB193B130E02095309550
:1019500020743327A90123E0559547952A95E1F78F
:10196000292F30E020953095207133273595279524
:1019700035952795242B8095807F822B0895FC0137
:1019800021912EBD9C5F21910DB407FEFDCF2EBD90
:10199000E817F907C1F70DB407FEFDCF0895CF9200
:1019A000DF92EF92FF920F931F93CF93E82FF0E017
:1019B000E154F44FC491E62FF0E0603330F4E35685
:1019C000F54FE4910E2F10E006C0EE0FFF1FE35617
:1019D000F64F059114916801E12CF12C60E074E25E
:1019E00084EF90E0A70196010E94441FBA01A9016B
:1019F00041505109610971094115510581E068079C
:101A0000710580F060E970ED83E090E0A701960138
:101A10000E94441FBA01A90141505109610971098D
:101A200083E001C081E0C130C9F0C33031F590914D
:101A30009100987F892B8093910050939900409357
:101A4000980010930D0300930C0381E080930B0327
:101A5000809171008260809371000FC0909181002D
:101A6000987F892B80938100509389004093880050
:101A700080916F00826080936F00CF911F910F91D2
:101A8000FF90EF90DF90CF9008951F920F920FB6C6
:101A90000F9211242F933F938F939F93AF93BF93F4
:101AA000EF93FF938091DA02882309F44DC080916F
:101AB000D6029091D702A091D802B091D902892B79
:101AC0008A2B8B2B51F180912203E0912303F0911B
:101AD00024039081892780838091D6029091D70238
:101AE000A091D802B091D902181619061A061B0641
:101AF000A4F58091D6029091D702A091D802B0911E
:101B0000D9020197A109B1098093D6029093D70217
:101B1000A093D802B093D90220C01092DA0280912B
:101B20006F008D7F80936F0090912203E0912303DB
:101B3000F09124038081282F30E0892F90E0809558
:101B400090958223932308C080912203E091230380
:101B5000F0912403908189278083FF91EF91BF91B9
:101B6000AF919F918F913F912F910F900FBE0F904A
:101B70001F901895E82FF0E0E154F44FE491E13024
:101B800019F0E33069F0089580916F008D7F8093A4
:101B90006F0090912203E0912303F091240308C089
:101BA00010920B0390911F03E0912003F091210309
:101BB0008081282F30E0892F90E0809590958223B6
:101BC0009323808308951F920F920FB60F921124D2
:101BD0002F933F934F935F936F937F938F939F9335
:101BE000AF93BF93EF93FF9380910B03882349F04A
:101BF00080911F03E0912003F091210390818927B8
:101C000080838091D502882309F493C080910703D3
:101C100090910803A0910903B0910A03892B8A2BA4
:101C20008B2B09F486C08091070390910803A09143
:101C30000903B0910A030197A109B1098093070331
:101C400090930803A0930903B0930A03892B8A2B6E
:101C50008B2B09F06EC0E0910503F0910603BF01E4
:101C60006F5F7F4F70930603609305034491942F39
:101C7000907F842F8F70903819F40E94BA0DEBCFAB
:101C8000903981F43296F0930603E0930503FB014B
:101C90006491909125038917F0F667FDDCCF0E94CF
:101CA000CF0CD9CF903E29F4109206031092050371
:101CB000D2CF903F19F41092D5023BC097FDCBCF05
:101CC0003296F0930603E0930503FB01249130E084
:101CD000342BA0910C03B0910D030E94851F6C5012
:101CE0007E4F8F4F9F4F28EE33E040E050E00E9440
:101CF000631F209307033093080340930903509315
:101D00000A038091070390910803A0910903B09101
:101D10000A03892B8A2B8B2B61F481E090E0A0E0F1
:101D2000B0E08093070390930803A0930903B09356
:101D30000A03FF91EF91BF91AF919F918F917F9196
:101D40006F915F914F913F912F910F900FBE0F9028
:101D50001F9018956038710518F54034510500F54D
:101D6000A42FA695A695A695B0E047705527B695E1
:101D7000BA2FAA27B795A7956A0F7B1FFC01E60F1C
:101D8000F71F81E090E001C0880F4A95EAF722230F
:101D900019F09489892B03C0809594898923848BB9
:101DA00008952F923F924F925F926F927F928F92FF
:101DB0009F92AF92BF92CF92DF92EF92FF920F93DA
:101DC0001F93CF93DF93CDB7DEB72A970FB6F89462
:101DD000DEBF0FBECDBF6A3091F4FC01E85EFB4F61
:101DE000408132972081318158E0459F200D311D7F
:101DF000112431832083329711821082C1C06D304B
:101E000009F4BEC09A878987885E9B4F9C838B8329
:101E1000DC012C90E985FA85EA5EFB4F60807180D9
:101E2000E985FA85EC5EFB4FFA83E9830081118135
:101E300000381105D4F0AB81BC812C91422F50E0C9
:101E4000E981FA8180819181F6E02F9F800D911DBB
:101E50001124A981BA818D939C93E985FA85E75E67
:101E6000FB4F208121115EC08BC0B0E46B16710462
:101E700014F7C801E5E02E9E800D911D112418165F
:101E80001906CCF6422C512CC301F8E02F9E800D90
:101E9000911D11241816190674F655E0659F9001DE
:101EA00011243F832E83E12CF12C85E0E816F10408
:101EB00041F0EE81FF81EE0DFF1DE350FB4F3490AA
:101EC00001C0312C630138E0932D91709D8348014E
:101ED000882D801B8215B0F456018A2D8C1982152D
:101EE00068F42D81A501B40189859A8538870E94FF
:101EF000AA0EAFEFAA1ABA0A3885EFCFBFEF8B1A36
:101F00009B0AE6CF36943150C40CD51C3111DCCF7E
:101F1000EFEFEE1AFE0A040D151DF6E0EF16F104C0
:101F200021F689CF6AEF64039001659F300D11247B
:101F300020583F4F281739071CF5A985BA85ED9120
:101F4000FC9111970190F081E02D6AE0CD012A9675
:101F50000FB6F894DEBF0FBECDBFDF91CF911F91BA
:101F60000F91FF90EF90DF90CF90BF90AF909F9038
:101F70008F907F906F905F904F903F902F9009943B
:101F80002A960FB6F894DEBF0FBECDBFDF91CF917A
:101F90001F910F91FF90EF90DF90CF90BF90AF9087
:101FA0009F908F907F906F905F904F903F902F9079
:101FB0000895CF93DF9390912503923009F46EC07A
:101FC000C82F292F30E0F901E154F44FD491F901E1
:101FD000E456F84F80839F5F9093250361E00E9451
:101FE000BE0AD13019F0D33039F158C010928000B8
:101FF000109281008091810088608093810080919F
:1020000081008160809381008C2F90E0FC01E0567C
:10201000F44FE491F0E0EE0FFF1FEE56F44F2591E0
:1020200034913093240320932303FC01ED58F44FA3
:1020300084918093220332C01092900010929100FC
:1020400080919100886080939100809191008160DF
:10205000809391008C2F90E0FC01E056F44FE491C6
:10206000F0E0EE0FFF1FEE56F44F259134913093C0
:10207000210320932003FC01ED58F44F84918093B9
:102080001F0380912503882321F06CE380E00E94E8
:10209000CF0C80E0DF91CF910C94BA0DDF91CF91FE
:1020A000089520E08AE893E0B22FB111BFEFFC0160
:1020B0000024B193B193B193B1930394D1F70895F0
:1020C000009769F0FC0101900020E9F73197AF011A
:1020D000481B590BBC0186E793E00C94AB0680E0EB
:1020E00090E008954F925F926F927F928F929F92AD
:1020F000AF92BF92CF92DF92EF92FF920F931F9316
:10210000CF93DF93EC018B01442ECB018C1B9D0BF5
:1021100097FF03C091958195910955245394813877
:1021200091053CF4512CC80100E810E0E12CF12CA1
:102130000FC00C171D0734F07E0180E890E0C0E06E
:10214000D0E006C078018E0180E090E0C0E8D0E0E9
:1021500038016E187F085C01AC1ABD0AB7FE03C0D7
:10216000B194A194B108630177FE03C02FEFC21AA6
:10217000D20AD594C794C817D90714F08FEF01C0BD
:1021800081E0882E880F99080E151F05C4F0242DB4
:10219000552019F0A701BE0102C0AE01B70186E7C4
:1021A00093E00E94AA0ECA18DB08D7FE04C0C80D2F
:1021B000D91DC60CD71C8FEFE81AF80AE5CFDF91BE
:1021C000CF911F910F91FF90EF90DF90CF90BF9034
:1021D000AF909F908F907F906F905F904F900895F9
:1021E0000F931F93CF93DF938C01C0E0D0E0F801F1
:1021F000EC0FFD1F6491662371F0E0917603F0917E
:1022000077030190F081E02D86E793E00995892B13
:1022100011F02196ECCFCE01DF91CF911F910F915C
:1022200008950F931F93CF93DF93C6E2D3E0E88125
:10223000F9810190F081E02D682FCE0109958C0184
:10224000E881F9810280F381E02D42E050E06EECFC
:1022500072E0CE010995800F911FDF91CF911F9100
:102260000F910895FC0180911E03811103C08FEF2F
:102270009FEF08959FB7F89482E08093E900209142
:10228000F20030E01216130614F421E030E02115BC
:10229000310559F0289884E680931D038091F10060
:1022A00080838091F200882319F09FBFC9010895AF
:1022B0008BE68093E800F9CF8091940781110DC0DF
:1022C00082E08093900784E08093910710929307B7
:1022D0001092920781E08093940780E997E0089537
:1022E000CF93DF9300D000D01F92CDB7DEB77894A4
:1022F00084B5826084BD84B5816084BD85B582600B
:1023000085BD85B5816085BD80916E0081608093BB
:102310006E00109281008091810082608093810024
:102320008091810081608093810080918000816034
:1023300080938000809191008260809391008091D1
:1023400091008160809391008091900081608093E2
:1023500090008091C10084608093C1008091C10091
:1023600082608093C1008091C10081608093C10030
:102370008091C30081608093C3008091C00082601F
:102380008093C0008091C20081608093C2008091E0
:102390007A00846080937A0080917A0082608093D2
:1023A0007A0080917A00816080937A0080917A002F
:1023B000806880937A0010921E031092D4021092CB
:1023C000D3028091D70081608093D70080EA809308
:1023D000D80089B5806189BD89B5826089BD09B49D
:1023E00000FEFDCF61E070E080E090E00E94920B83
:1023F0008091D8008F7C80618093D8008091E0002C
:10240000807F8093E0008091E1008E7E8093E100E8
:102410008DE08093E200559A209AEEEFFFE78591D8
:1024200094918B3F9C4D19F481E08093D2021FB7A9
:10243000F8948091DC02811127C0E1EBFBE08491EC
:10244000E4E8FBE09491E82FF0E0EE0FFF1FEA5480
:10245000FE4FA591B491EC91E92321F461E081E173
:102460000E945B0A61E081E10E94BE0A8CB5806136
:102470008CBD8CB580648CBD61E08FE00E94BE0A8B
:1024800061E080E10E94BE0A8091DC028F5F809350
:10249000DC021FBF01ED11E0F801849131966491D7
:1024A000882329F00E5F1F4F0E94BE0AF5CF61E01E
:1024B00086E00E945B0A61E070E080E090E00E94AC
:1024C000920B60E086E00E945B0A6AE070E080E0C8
:1024D00090E00E94920B61E086E00E945B0AECEAC9
:1024E000FBE0E491F0E0EE0FFF1FEE56F44F859114
:1024F00094919093E2028093E102EFE7FBE0E49194
:10250000E093E002E4EAFBE0E491F0E0EE0FFF1F6D
:10251000EE56F44F859194919093DF028093DE0202
:10252000E7E7FBE0E491E093DD028CB58C7F8CBDA6
:102530008DB581608DBDE091E102F091E202908164
:102540008091E002982B9083A091DE02B091DF028F
:102550002C919091DD02909592239C93908180958F
:1025600089238083E4ECF1E021E0E13DF20749F0CA
:1025700084918EBD00000DB407FEFDCF8EB531965F
:10258000F3CFE091DE02F091DF0290818091DD02D5
:10259000892B8083E091E102F091E20290818091A9
:1025A000E00280958923808380916400816080931C
:1025B0006400809164008260809364008091640074
:1025C00080688093640080916400806480936400DC
:1025D000809165008160809365000E94A20C87FF56
:1025E0001AC080E094E01EBC00000DB407FEFDCFD1
:1025F0002EB50197C1F760E070E08AE00E94FA0A08
:1026000060E070E08BE00E94FA0A60E070E089E030
:102610000E94FA0AFFCF4EEE5FEF5B834A8318E118
:10262000412E88248A94912C08E010E0842D5A8150
:10263000851BB401681B71098AE00E94FA0A6FEFDA
:1026400070E08BE00E94FA0A6FEF70E089E00E9470
:10265000FA0A0E9451105A8060EF5616A4F48AE8D4
:1026600093E00E94BF0C6BE170E080E090E00E947C
:10267000920B70EF571265C06AEF70E080E090E057
:102680000E94920B5EC02A813B8137FF03C03195C7
:1026900021953109277033278A819B8197FD079601
:1026A000B3E095958795BA95E1F72A803B8037FE90
:1026B00005C00197A801421B530B9A017C01F694B7
:1026C000FE2CEE24F794E79440E050E03801621AC3
:1026D000730AB70160587F4F5B018F3F7FEF970709
:1026E00044F40196485A5F4F7501403B510589F704
:1026F000B6CFD701A25EBB4F60E070E08F3FEFEF37
:102700009E0709F421C7FB01E40FF51FEA5FFE4FA6
:10271000E4916D01CA18DB08CE0CDF1CF0E01F014C
:10272000022E02C0220C331C0A94E2F73D822C8256
:10273000F6013080EC81FD81E3291F01F601208242
:1027400003C72A813B812F5F3F4F3B832A83293177
:10275000310509F06BCF6EEE72E080E090E00E94F0
:10276000920B6FEF70E08AE00E94FA0A6FEF70E060
:102770008BE00E94FA0A6FEF70E089E00E94FA0A8B
:1027800085E00E94D90F8DE00E94D90F1092D502EA
:1027900082E090E00E942E1F882369F080916400FF
:1027A000877F8093640080916500877F80936500B8
:1027B00081E08093DB0284E680937C038AE080934F
:1027C0007F038AE893E00E94BF0C01E010E0F8E18B
:1027D0006F2E712C1F9280E18F931F928DE28F9349
:1027E000A2E9B2E0BF93AF93A3E0B3E0BF93AF938E
:1027F0000E948D1C0E94511010928B0710928A0724
:1028000010928D0710928C070FB6F894DEBF0FBEA2
:10281000CDBFE0910103F0910203EF30F10508F024
:102820001FC6EA5AFF4F0C94821C109200031092AC
:10283000FF02809111019091120101979093120172
:1028400080931101892B31F482E090E09093020390
:102850008093010343E050E050938B0740938A0735
:1028600087EE94E00E94F01063E170E070938B07B4
:1028700060938A078CE090E090938D0780938C079B
:1028800087ED94E00E94F010AEE2B0E0B0938B07C9
:10289000A0938A0770928D0760928C0780ED94E078
:1028A0000E94F010E3E0F0E0F0938B07E0938A07DA
:1028B000E4E22E2E312C30928D0720928C078AEB89
:1028C00094E00E94F01041E066E370E086E390E05F
:1028D0000E94721010928B0710928A0728E330E052
:1028E00030938D0720938C078091110190911201F4
:1028F0008C3291401CF489E491E002C081E691E0C1
:102900000E9460100E94A20C83FFAAC58091100152
:10291000811198C5A5C588E090E09093000380934D
:10292000FF022091FD023091FE0282E190E090933F
:102930008B0780938A07263031056CF085E090E0A4
:10294000821B930B73E0880F991F7A95E1F79093A0
:102950008D0780938C0783E494E00E94F0100E941E
:10296000A20C83FF1FC0809110018823D9F08091B1
:10297000FD029091FE029C012E5F3F4F30930203B7
:10298000209301038630910509F0F9C58DE090E0B0
:1029900090930203809301031092FE021092FD02B5
:1029A0001092100141E066E370E086E390E00E943F
:1029B000721040E065E370E085E390E00E947210E1
:1029C00010928B0710928A0748E350E050938D07CE
:1029D00040938C078EE691E036C01092000310926F
:1029E000FF0289E791E00E9460100E94A20C83FF21
:1029F00004C086E891E00E9460100E94A20C82FF51
:102A000004C081E991E00E9460100E94A20C87FF3F
:102A100004C08CE991E00E9460100E94A20C85FF26
:102A200004C088EA91E00E9460100E94A20C86FF18
:102A300004C086EB91E00E9460100E94A20C84FF0B
:102A40000FC585EC91E00E9460100AC5109200034A
:102A50001092FF0220910F01822F022E000C990B81
:102A60009F932F9383ED91E09F938F9365EEE62ED6
:102A700062E0F62EFF92EF920E948D1CC7010E9429
:102A8000601020910F01822F022E000C990B9F9352
:102A90002F9382EE91E09F938F93FF92EF920E948B
:102AA0008D1CC7010E9460100E94A20C0FB6F89402
:102AB000DEBF0FBECDBF87FF04C080911001811122
:102AC00064C50E94A20C84FF04C080911001811192
:102AD00064C580910D0190910E0197FF04C0109282
:102AE0000E0110920D010E94A20C82FF04C0809181
:102AF000100181115AC541E06EE270E08EE290E073
:102B00000E94721010928B0710928A0780E390E067
:102B100090938D0780938C0789E294E018C484E039
:102B200090E0909300038093FF0286EE93E00E9472
:102B3000F0100E94A20C83FF11C08091100181113E
:102B40003FC50CC0823091050CF047C5892B31F48C
:102B500088E090E090930203809301030E94A20C0E
:102B600082FF04C080911001811143C541E066E3FA
:102B700070E086E390E00E94721010928B07109232
:102B80008A07A8E3B0E0B0938D07A0938C0788EA8A
:102B900092E059CF85E090E0909300038093FF028C
:102BA00080910701811103C086E491E002C082E4B4
:102BB00091E09F938F9381EF91E09F938F9385EEA8
:102BC00092E09F938F930E948D1C85EE92E00E946D
:102BD00060100F900F900F900F900F900F908091BA
:102BE0000801811103C086E491E002C082E491E013
:102BF0009F938F9386E092E09F938F9385EE92E070
:102C00009F938F930E948D1C85EE92E00E9460102E
:102C10000F900F900F900F900F900F9080910901DF
:102C2000811103C086E491E002C082E491E09F93A9
:102C30008F938BE192E09F938F9385EE92E09F9329
:102C40008F930E948D1C85EE92E00E9460100F9081
:102C50000F900F900F900F900F9080910A018111AB
:102C600003C086E491E002C082E491E09F938F93D9
:102C700080E392E09F938F9385EE92E09F938F93F2
:102C80000E948D1C85EE92E00E9460100F900F90C4
:102C90000F900F900F900F9080910B01811103C046
:102CA00086E491E002C082E491E09F938F9385E4F3
:102CB00092E09F938F9385EE92E09F938F930E9473
:102CC0008D1C85EE92E00E9460100E94A20C0F9075
:102CD0000F900F900F900F900F9083FF04C0809182
:102CE0001001811191C40E94A20C82FF04C0809146
:102CF0001001811196C4609107018AE00E945B0A6D
:102D0000609108018BE00E945B0A6091090189E0F3
:102D10000E945B0A60910A0181E10E945B0A609156
:102D20000B018EE10E945B0A41E066E370E086E3FE
:102D300090E00E94721010928B0710928A07E8E3CD
:102D4000F0E0F0938D07E0938C0780ED93E0FFC2F5
:102D5000109200031092FF022091050130910601AC
:102D60008091030190910401A901243631051CF4DE
:102D70004B5F5F4F02C04A53510950938B074093FA
:102D80008A07863091052CF0059790938D078093E4
:102D90008C07809104018F93809103018F933F935F
:102DA0002F938AE592E09F938F9385EE92E09F9315
:102DB0008F930E948D1C85EE92E00E946010E0903F
:102DC0000301F09004015701F1E0AF1AB108C0907F
:102DD0000501D090060121E0A501B60186E793E048
:102DE0000E94AA0E460121E0821A910821E0A70163
:102DF000B40186E793E00E94AA0E21E0A701B60184
:102E000086E793E00E94AA0EB6016F5F7F4F21E034
:102E1000A70186E793E00E94AA0EA7014F5F5F4FCC
:102E200021E0B60186E793E00E94AA0E0E94A20C60
:102E30000FB6F894DEBF0FBECDBF85FF04C08091F2
:102E400010018111F9C30E94A20C86FF04C0809179
:102E500010018111F8C30E94A20C87FF04C0809169
:102E600010018111FCC30E94A20C84FF04C0809158
:102E700010018111FBC30E94A20C82FFF1C280915C
:102E800010018111FFC3ECC2109200031092FF02E7
:102E900080910E018F9380910D018F9383E692E0D4
:102EA0009F938F9385EE92E09F938F930E948D1C4A
:102EB00085EE92E00E9460100E94A20C0F900F908D
:102EC0000F900F900F900F9087FF0BC080910D0116
:102ED00090910E01019690930E0180930D01109236
:102EE00010010E94A20C84FF0BC080910D019091F3
:102EF0000E01019790930E0180930D011092100125
:102F000080910D0190910E0197FF04C010920E0167
:102F100010920D010E94A20C82FF04C0809110014A
:102F20008111BBC30E94A20C83FF55C0E0900D012C
:102F3000F0900E0181E08093DA021701412C512CB0
:102F400060E072E18AE790E0A20191010E94441FD3
:102F500049015A0161E0861A9108A108B10881145B
:102F6000910471E0A706B10488F068E478EE81E08E
:102F700090E0A20191010E94441F49015A0181E0A1
:102F8000881A9108A108B10893E001C091E08091EE
:102F90008100887F892B809381009701220F331F46
:102FA000A8E2B0E00E94851F28EE33E040E050E048
:102FB0000E94631F90928900809288002093D6021D
:102FC0003093D7024093D8025093D90280916F007A
:102FD000826080936F0041E06EE270E08EE290E0EC
:102FE0000E94721010928B0710928A0780E390E083
:102FF00090938D0780938C0788EA93E0A8C1109284
:1030000000031092FF02809102018F9380910101D1
:103010008F9382E792E09F938F9385EE92E09F9348
:103020008F930E948D1C85EE92E00E94601080912B
:103030000101909102010E942E1F0F900F900F909E
:103040000F900F900F9080FD02C070E301C071E3FC
:1030500081FD02C060E301C061E382FD02C050E374
:1030600001C051E383FD02C040E301C041E384FDA0
:1030700002C030E301C031E385FD02C020E301C09E
:1030800021E386FD02C090E301C091E3881F8827F9
:10309000881F805D1F927F931F926F931F925F9393
:1030A0001F924F931F923F931F922F931F929F93B4
:1030B0001F928F9380E892E09F938F9385EE92E02A
:1030C0009F938F930E948D1C85EE92E00E9460106A
:1030D0000E94A20C0FB6F894DEBF0FBECDBF82FFD8
:1030E00004C0809110018111E3C20E94A20C87FFED
:1030F00004C0809110018111E8C20E94A20C84FFDB
:1031000004C0809110018111ECC280910101909165
:10311000020197FF06C08FEF93E090930201809326
:10312000010180910101909102018115944024F0E8
:10313000109202011092010141E06EE270E08EE215
:1031400090E00E94721010928B0710928A0780E321
:1031500090E090938D0780938C0787E992E073CC81
:10316000109200031092FF028EE693E00E94F0108E
:103170000E94A20C82FF04C0809110018111BDC287
:103180000E94A20C83FF11C0809110018111C2C264
:103190000CC08BE090E090930203809301031092A7
:1031A000FE021092FD021092100141E066E370E011
:1031B00086E390E00E94721010928B0710928A07AB
:1031C00048E3242E312C30928D0720928C078DE518
:1031D00093E0BDC0109200031092FF0286E193E0DD
:1031E0000E94F0100E94A20C83FF2BC0809110015E
:1031F0008111C1C226C0C7010E942E1F882321F061
:1032000060E0C7010E94361F8091E3029091E402C2
:1032100001969093E4028093E302E090E302F09041
:10322000E402E11424E0F20634F38BE090E09093A2
:103230000203809301031092FE021092FD0210928D
:1032400010010E94A20C82FF04C080911001811124
:10325000ADC241E066E370E086E390E00E94721048
:1032600010928B0710928A0748E350E050938D0725
:1032700040938C0785E093E06AC01092000310929F
:10328000FF0281EB92E00E9460100E94A20C83FF7B
:1032900004C080911001811196C241E066E370E0A4
:1032A00086E390E00E94721010928B0710928A07BA
:1032B00068E370E070938D0760938C0781E691E07E
:1032C000C2CB109200031092FF0286EA92E00E94A5
:1032D000F0100E94A20C83FF1FC080911001811189
:1032E0007DC21AC086E293E00E946A07682F8E367C
:1032F00009F093C286E293E00E94F706892B91F7CA
:103300008BE090E090930203809301031092FE0201
:103310001092FD02109210010E94A20C82FF04C0C4
:1033200080911001811192C241E066E370E086E372
:1033300090E00E94721010928B0710928A0788E327
:1033400090E090938D0780938C0788E892E00E942C
:10335000F01086C0109200031092FF0287E292E004
:103360000E94F01086E293E00E94F706892B61F03C
:1033700086E293E00E946A07F82E0E941111809164
:103380000001F812F0920001E0917603F0917703CA
:103390000190F081E02D6091000186E793E00995AE
:1033A0003DC0109200031092FF02A3E0B0E0B09382
:1033B0008B07A0938A0781E192E00E94F010E3E17D
:1033C000F0E0F0938B07E0938A073CE0232E312C4A
:1033D00030928D0720928C0781E092E00E94F010DD
:1033E0002EE230E030938B0720938A0770928D078E
:1033F00060928C078AEF91E00E94F01043E050E069
:1034000050938B0740938A0764E270E070938D07B6
:1034100060938C0784EE91E00E94F0100E94A20C51
:1034200082FFA4CB80911001882309F49FCB1093D5
:103430000203009301031092FE021092FD0210920B
:10344000100194CB109210011092FE021092FD0216
:1034500010930203009301031092120110921101C4
:103460008091FF0290910003892B09F445C080915F
:10347000FD029091FE0210928B0710928A0786300F
:10348000910534F423E0880F991F2A95E1F702C0D3
:1034900088E290E090938D0780938C0783E093E01F
:1034A0000E9460100E94A20C87FF04C0809110014E
:1034B0008111D9C10E94A20C84FF04C08091100127
:1034C0008111DDC18091FF02909100032091FD02E6
:1034D0003091FE022817390724F01092FE02109254
:1034E000FD022091FD023091FE0237FF05C00197D9
:1034F0009093FE028093FD0280911001811118C00B
:103500000E94A20C87FD14C00E94A20C84FD10C072
:103510000E94A20C85FD0CC00E94A20C86FD08C072
:103520000E94A20C83FD04C00E94A20C82FFB3C1C2
:103530008AE893E00E94BF0C80E090E0892B09F4B8
:1035400049C90E94000043C92115310581F0FB01E2
:10355000E40FF51FEA5FFE4FE491F0E0062C02C095
:10356000F595E7950A94E2F7DC90ED29EC936F5F0F
:103570007F4F11966835710509F0C0C8B2C807972A
:1035800009F00ACA8EE090E003CA80910F018F5FB4
:1035900080930F011092100194CA80910F01815005
:1035A00080930F011092100194CA109302030093AC
:1035B00001031092FE021092FD02109210019BCAAC
:1035C000109210018091FD029091FE0281309105D0
:1035D00009F0B8CA89E090E0BDCA8230910519F4BB
:1035E0008CE090E0B7CA039709F0B8CA8AE090E08F
:1035F000B1CA1093020300930103109210011092BC
:10360000FE021092FD02B2CA10921001E091FD027A
:10361000F091FE02E95FFE4F908181E0892780836F
:1036200062CB1092100110930203009301031092D9
:10363000FE021092FD025FCB1092100190920601E3
:103640008092050100CC10921001809105019091AB
:10365000060101969093060180930501FCCB109220
:103660001001B0920401A0920301FDCB1092100151
:10367000809103019091040101969093040180933D
:103680000301F9CB10921001109302030093010380
:103690001092FE021092FD02E3CE109302030093FB
:1036A00001031092FE021092FD02109210013ACC1A
:1036B00084E090E090930203809301031092FE0255
:1036C0001092FD021092100110CD80910101909195
:1036D0000201019690930201809301011092100162
:1036E0000CCD10921001809101019091020101977F
:1036F000909302018093010108CD84E090E09093C3
:103700000203809301031092FE021092FD021092B8
:10371000100136CD0E94511010928B0710928A072B
:1037200070928D0760928C0787EB92E00E94601088
:103730008AE893E00E94BF0C64EF71E080E090E0C3
:103740000E94920B80E190E09093E4028093E30268
:103750008091E3029091E4028115E4E09E070CF071
:1037600018CD0E942E1F0E9411118091E3029091AA
:10377000E4020196E9CF0E94511010928B0710923B
:103780008A0770928D0760928C0782EC92E00E940B
:1037900060108AE893E00E94BF0C64EF71E080E063
:1037A00090E00E94920B80E190E033CD84E090E0C5
:1037B00090930203809301031092FE021092FD0287
:1037C0001092100146CD1093020300930103109252
:1037D000FE021092FD02109210015FCD0E94511066
:1037E00010928B0710928A0770928D0760928C0757
:1037F00089E992E00E94F0108AE893E00E94BF0CF1
:1038000064EF71E080E090E00E94920B80E190E034
:103810009093E4028093E3026DCDE090E302F09098
:10382000E402E11474E0F7060CF064CDC70169838B
:103830000E942E1F6981681719F0C7010E94361F68
:103840008091E3029091E4020196E2CF84E090E05F
:1038500090930203809301031092FE021092FD02E6
:103860001092100161CD8091FD029091FE020197AE
:103870009093FE028093FD02109210011BCE809166
:10388000FD029091FE0201969093FE028093FD024C
:103890001092100117CE81E08093100149CEE6E22C
:1038A000F3E01382128288EE93E0A0E0B0E084831C
:1038B0009583A683B7838EE291E0918380838FEF17
:1038C0009FEF95878487E6E7F3E0138212828EE309
:1038D00091E0918380838CE3868380E181871086E9
:1038E000178216861786108A118A128A10928B0701
:1038F00010928A0710928D0710928C0781E08093B6
:103900008E070895EE0FFF1F0590F491E02D0994A6
:1039100081E090E0F8940C94CB1FAEE0B0E0E3E9D6
:10392000FCE10C94A21F0D891E8986E08C831A830A
:1039300009838FEF9FE79E838D83AE01475E5F4FC4
:103940006F89788DCE0101960E94B01C2F81388539
:10395000F801E20FF31F10822E96E4E00C94BE1FD4
:10396000ACE0B0E0E6EBFCE10C94941F7C016B0151
:103970008A01FC0117821682838181FFBDC1CE01BD
:1039800001964C01F7019381F60193FD859193FF18
:1039900081916F01882309F4ABC1853239F493FD1D
:1039A000859193FF81916F01853229F4B70190E0F1
:1039B0000E94981EE7CF512C312C20E02032A0F439
:1039C0008B3269F030F4803259F0833269F420612F
:1039D0002CC08D3239F0803339F4216026C022604A
:1039E000246023C0286021C027FD27C030ED380F98
:1039F0003A3078F426FF06C0FAE05F9E300D1124BD
:103A0000532E13C08AE0389E300D1124332E2062CD
:103A10000CC08E3221F426FD6BC1206406C08C36AA
:103A200011F4206802C0883641F4F60193FD8591B7
:103A300093FF81916F018111C1CF982F9F7D955484
:103A4000933028F40C5F1F4FFFE3F9830DC08336DA
:103A500031F0833771F0833509F05BC022C0F80183
:103A6000808189830E5F1F4F44244394512C54015D
:103A700015C03801F2E06F0E711CF801A080B18012
:103A800026FF03C0652D70E002C06FEF7FEFC50118
:103A90002C870E948D1E2C0183012C852F77222ECE
:103AA00017C03801F2E06F0E711CF801A080B180E0
:103AB00026FF03C0652D70E002C06FEF7FEFC501E8
:103AC0002C870E94821E2C012C852068222E8301C7
:103AD00023FC1BC0832D90E048165906B0F4B701B3
:103AE00080E290E00E94981E3A94F4CFF50127FC02
:103AF000859127FE81915F01B70190E00E94981E99
:103B000031103A94F1E04F1A51084114510471F701
:103B1000E5C0843611F0893639F5F80127FF07C072
:103B200060817181828193810C5F1F4F08C0608129
:103B30007181072E000C880B990B0E5F1F4F2F769B
:103B4000722E97FF09C090958095709561957F4F73
:103B50008F4F9F4F2068722E2AE030E0A4010E9410
:103B6000D01EA82EA81844C0853729F42F7EB22E67
:103B70002AE030E025C0F22FF97FBF2E8F36C1F04A
:103B800018F4883579F0B4C0803719F0883721F0FF
:103B9000AFC02F2F2061B22EB4FE0DC08B2D8460DC
:103BA000B82E09C024FF0AC09F2F9660B92E06C008
:103BB00028E030E005C020E130E002C020E132E042
:103BC000F801B7FE07C060817181828193810C5F2B
:103BD0001F4F06C06081718180E090E00E5F1F4F33
:103BE000A4010E94D01EA82EA818FB2DFF777F2EBF
:103BF00076FE0BC0372D3E7FA51450F474FE0AC02C
:103C000072FC08C0372D3E7E05C0BA2C372D03C08C
:103C1000BA2C01C0B52C34FF0DC0FE01EA0DF11D18
:103C20008081803311F4397E09C032FF06C0B3941D
:103C3000B39404C0832F867809F0B39433FD13C086
:103C400030FF06C05A2CB31418F4530C5B18B32C75
:103C5000B31468F4B70180E290E03C870E94981E9C
:103C6000B3943C85F5CFB31410F43B1801C0312C4C
:103C700034FF12C0B70180E390E03C870E94981E99
:103C80003C8532FF17C031FD03C088E790E002C0D9
:103C900088E590E0B7010CC0832F867859F031FF9A
:103CA00002C08BE201C080E237FD8DE2B70190E0F7
:103CB0000E94981EA51438F4B70180E390E00E949A
:103CC000981E5A94F7CFAA94F401EA0DF11D808151
:103CD000B70190E00E94981EA110F5CF332009F49F
:103CE00051CEB70180E290E00E94981E3A94F6CF40
:103CF000F7018681978102C08FEF9FEF2C96E2E15A
:103D00000C94B01FFC010590615070400110D8F771
:103D1000809590958E0F9F1F0895FC016150704013
:103D200001900110D8F7809590958E0F9F1F0895F0
:103D30000F931F93CF93DF93FB01238121FD03C0DA
:103D40008FEF9FEF28C022FF16C046815781248144
:103D500035814217530744F4A081B1819D012F5F43
:103D60003F4F318320838C93268137812F5F3F4FD4
:103D70003783268310C0EB01092F182F0084F185AB
:103D8000E02D0995892BE1F68E819F8101969F8315
:103D90008E83812F902FDF91CF911F910F910895E6
:103DA000FA01AA27283051F1203181F1E8946F936C
:103DB0006E7F6E5F7F4F8F4F9F4FAF4FB1E03ED012
:103DC000B4E03CD0670F781F891F9A1FA11D680FB0
:103DD000791F8A1F911DA11D6A0F711D811D911DE3
:103DE000A11D20D009F468943F912AE0269F112458
:103DF0003019305D3193DEF6CF010895462F4770BC
:103E0000405D4193B3E00FD0C9F7F6CF462F4F7016
:103E1000405D4A3318F0495D31FD4052419302D074
:103E2000A9F7EACFB4E0A69597958795779567951A
:103E3000BA95C9F700976105710508959B01AC011A
:103E40000A2E06945795479537952795BA95C9F741
:103E5000620F731F841F951FA01D0895F999FECF4F
:103E600092BD81BDF89A992780B50895262FF999BA
:103E7000FECF1FBA92BD81BD20BD0FB6F894FA9A4D
:103E8000F99A0FBE01960895052E97FB1EF4009433
:103E90000E945B1F57FD07D00E94631F07FC03D0E1
:103EA0004EF40C945B1F50954095309521953F4FF3
:103EB0004F4F5F4F089590958095709561957F4F16
:103EC0008F4F9F4F0895A1E21A2EAA1BBB1BFD0125
:103ED0000DC0AA1FBB1FEE1FFF1FA217B307E407E9
:103EE000F50720F0A21BB30BE40BF50B661F771F41
:103EF000881F991F1A9469F7609570958095909521
:103F00009B01AC01BD01CF010895A29FB001B39FF9
:103F1000C001A39F700D811D1124911DB29F700DD2
:103F2000811D1124911D08952F923F924F925F920F
:103F30006F927F928F929F92AF92BF92CF92DF92B9
:103F4000EF92FF920F931F93CF93DF93CDB7DEB71E
:103F5000CA1BDB0B0FB6F894DEBF0FBECDBF0994B2
:103F60002A88398848885F846E847D848C849B8409
:103F7000AA84B984C884DF80EE80FD800C811B8117
:103F8000AA81B981CE0FD11D0FB6F894DEBF0FBE46
:0A3F9000CDBFED010895F894FFCFB6
:103F9A0020100019001900010101010101C8006186
:103FAA0001B004FFFFFFFF00E10000000000000174
:103FBA0000000000C1808100000000000000D60659
:103FCA00CC0BF7066A078807EC0600000000D10E42
:103FDA00AB064F6666004F6E005761697420666FC4
:103FEA007220627574746F6E20746573742E2E2E2F
:103FFA000028412920436F6E74696E756500284157
:10400A00292053656C65637400427574746F6E2061
:10401A00546573740A004120507265737365640AAB
:10402A00004220507265737365640A00555020502F
:10403A007265737365640A004C4546542050726574
:10404A00737365640A005249474854205072657375
:10405A007365640A00444F574E2050726573736546
:10406A00640A00496E74656765723A2020202564E7
:10407A000A004368617261637465723A2025630AB3
:10408A0000202020526564204C45443A20202020FC
:10409A00202025730A00202020477265656E204C77
:1040AA0045443A2020202025730A00202020426C13
:1040BA007565204C45443A202020202025730A00AB
:1040CA0020202052656365697665204C45443A2074
:1040DA002025730A002020205472616E736D697462
:1040EA00204C45443A2025730A002825642C2025B3
:1040FA006429004672657175656E63793A20256494
:10410A000A004C6F636174696F6E3A2025640A0075
:10411A00446174613A202563256325632563256319
:10412A00256325632563002855702F446F776E2910
:10413A00205363726F6C6C0A284229204261636BB8
:10414A0000446F6E65210053656E64696E672E2E9A
:10415A002E00436C656172696E672E2E2E000D0A61
:02416A00000053
:00000001FF
